:1000000000308A006D290000831685118312851146
:10001000A630F700F70B0A28000083168515A630D6
:10002000F700F70B11280000851583120034B30187
:100030003308073C031C372883168511831285116A
:10004000000000000314B20C031828288511292889
:100050008515831685111330F700F70B2D28000046
:1000600000008515000000008312B30A1828003430
:10007000B2013208073C031C5A28831685118312EB
:10008000851100000000831685150230F700F70B7C
:100090004728000085158312851950280310512820
:1000A0000314B30C2730F700F70B542800000000AE
:1000B000B20A39283308F80000343308350680398D
:1000C000B700B31F6828B209B309B20A0319B30A0B
:1000D000B51F6F28B409B509B40A0319B50AF801A8
:1000E000F901F701FA013508031D792834080319CD
:1000F00093281030B6000310B20DB30DF70DFA0DB2
:1001000035087A02031D862834087702031C8F28DD
:100110003408F702031CFA033508FA020314F80D39
:10012000F90DB60B7B280000B71F9B28F809F909C9
:10013000F80A0319F90A8A11E4288E30F700330807
:10014000F8003208F900FA01F808031DB12879080F
:10015000F800F9010830F702F808031DB128F7018B
:10016000B9280310F81BB828F90DF80DF703B128CA
:10017000F81300008A11E828A9010420CC30B2004D
:1001800017204430B2001720A908031DCB283820BF
:100190007808A900C4280420CC30B2001720BE3053
:1001A000B200172038207808AA0038207808AB0061
:1001B0002B08AD002A08AC002D08B3002C08B200B3
:1001C000B5011030B4005D287808B301B2009D2855
:1001D0007A08B1007908B0007808AF007708AE005F
:1001E0002E08F7002F08F8003008F9003108FA004F
:1001F0008A11A7298E30F7002908F7022A08F9008A
:100200002B08F800F917F708031911290310F9084A
:10021000031D0D29F80803191129F90CF80CF70B27
:100220000629AA1F1829F809F909F80A0319F90A71
:1002300000008A11B0292A08F8012902031823298D
:100240002908F7002F29F7010830AB00A90DF70D99
:100250002A0877020318F700F80DAB0B26298A113C
:10026000BF29F701F801290803102A18F707F70C2E
:10027000F80CAA18F707F70CF80C2A19F707F70C6F
:10028000F80CAA19F707F70CF80C2A1AF707F70C5D
:10029000F80CAA1AF707F70CF80C2A1BF707F70C4B
:1002A000F80CAA1BF707F70CF80C8A11C62929309D
:1002B0008400000803196B290130F800F701F70BDF
:1002C0005F29F80B5E294A30F700F70B652900001B
:1002D0000000800B5C298A11412A84011F308305AC
:1002E000603083168F001F129F121B0880399B00FD
:1002F00007309C001F129F121B0880399B0083123D
:100300001F109412831606118614061200308312F1
:100310009400831694000108C739083881008312BD
:1003200090010030F80092000030831692000730F0
:100330009C0005080330F700F70B9C291C0883126A
:100340000D1383169D018F010F088312BC287A08B4
:10035000AC007908AB007808AA007708A900FA2851
:100360007808A3002308093C031CBA292308A40029
:10037000A501C9292308A9000A30AA001B29780869
:10038000A5002508A9000A30AA003129780823020F
:10039000A400A7012708013C031C432AA708031D4A
:1003A000DB298316851083128510831605118312AD
:1003B00005152408A600270BE729831605118312CB
:1003C000051183168510831285142508A600260BB7
:1003D000EE2983168601F330831286002608023C3C
:1003E000031DF729831686014930831286002608EB
:1003F000033C031D002A83168601613083128600A8
:100400002608043C031D092A831686013330831213
:1004100086002608053C031D122A83168601253016
:10042000831286002608063C031D1B2A83168601BC
:100430000530831286002608073C031D242A8316F4
:100440008601F130831286002608083C031D2D2A00
:10045000831686010130831286002608093C031D9D
:10046000362A83168601213083128600A608031DD2
:100470003E2A831686018130831286000A30A90045
:0C0480005729A70ACA298316A529630082
:04400E00F83FFF3F39
:00000001FF
